:02000000392A9B
:0A00060000000000000008000800E0
:10001000103083120313FD00FD0B0C2800000800B4
:0400200000000800D4
:10002400083083120313FC002330FD00FD0B182855
:06003400FC0B1828080077
:10003A00032083120313851403208510032008006C
:02004A000800AC
:10004C008312031305148316051403200030831246
:10005C0005180130B9001D20831603130510032069
:04006C000800080080
:1000700083120313D71B3E2886113F288615571B72
:100080004328061144280615D71A482886104928FF
:100090008614571A4D2806104E2806143B1852286D
:1000A000051553280511851510208511D7195A28D3
:1000B00086115B28861557195F28061160280615DA
:1000C000D7186428861065288614571869280610E2
:1000D0006A2806143B186E2805156F28051185152A
:1000E000102085113B1C7628122077280820080054
:1000F0008316031305108312C00180303805F10008
:100100007108BD007108003A031D88280510892870
:1001100005141D2083120313B80D38104008073A48
:0C01200003199428C00A7D28080008007C
:10012C00831203133B105608D70038203B140800E9
:10013C0083120313B8018316051403208312C00124
:10014C00B80D38100518AC283810AD2838141D20FF
:10015C00831203134008073A0319B628C00AA628CD
:04016C00080008007F
:100170008312031305148514032005100320851032
:0601800003200800080046
:10018600831203130510032085140320051403208E
:040196000800080055
:10019A008312031333083704B80078202620831209
:1001AA0003133608F200F3017208BE00FF3035056A
:1001BA00F0003608F1000030F1057008BF0072083F
:1001CA00B80078202620831203133F08B80078204D
:0601DA00262008000800C9
:1001E0008316031305108510B820CD20B820831284
:1001F000031333083704B8003814782026208312FC
:100200000313B801BA019E20831203133A08203E5B
:10021000840038088000BA0A34083A020318162904
:1002200083160510831205101D200329831603135E
:0E0230000510831205141D20C32008000800CD
:10023E0083160313861706178616061606108610E3
:10024E00061186114130FC00EE30FD00FD0B2D290C
:10025E00FC0B2D29000010308312BC0006108614F2
:10026E0006158615861B3D290130BC00061B41294B
:10027E000430BC00861A45290730BC00061A4929ED
:10028E000A30BC0006148610861B4F290230BC00B3
:10029E00061B53290530BC00861A57290830BC00AE
:1002AE00061A5A29BC0186140611861B60290330D2
:1002BE00BC00061B64290630BC00861A682909306A
:1002CE00BC00061A6C290B30BC0006158611861B65
:1002DE0072290C30BC00061B76290D30BC00861A24
:1002EE007A290E30BC00061A7E290F30BC003C085D
:1002FE00103A031D85291030B20008003C08320662
:0E030E00031D8A2929293C08B20008000800B6
:10031C008316031305108510B820CD208312031308
:10032C00BA013403D2003A085202031CAC293A0831
:10033C00203E84000008B800782026208312031386
:10034C003A0852060319AC29BA0A9729C3200800A7
:02035C00080097
:10035E00831203135208013A031DB8298030D200CC
:10036E00CF295208023A031DBF29C030D200CF292F
:10037E005208033A031DC6299430D200CF295208E1
:10038E00043A031DCD29D430D200CF298030D200BB
:10039E005303F0005208F0077008D2007008D7001F
:1003AE0038203B10D5015508540784000008003A48
:1003BE000319E9295508540784000008D600962031
:0803CE00D50ADA293B140800EE
:1003D6008316031385110511061086100611861162
:1003E600831285110511861106118610061012203A
:1003F600122012208614061485151020851112204D
:1004060085151020851112208515102085111220C2
:1004160006108515102085111220851510208511CE
:100426008610861585151020851112208611061452
:1004360085151020851106108515102085111220AE
:10044600851510208511061485151020851112209A
:1004560006108515102085118615061586140614B6
:0C04660085151020851112203B140800A1
:10047200831603139B01811346308312A00052306E
:10048200A1004130A2004E30A3004330A400453009
:10049200A5005330A6004330A7004F30A8002030FB
:1004A200A9004930AA005430AB003930AC004430C6
:1004B200AD005030AE005830AF00B001EB2101303A
:1004C200D70038200C30D70038200230D20001305B
:1004D200D3002030D400AF210B30FB002630FC00CB
:1004E2005D30FD00FD0B732AFC0B732AFB0B732A94
:1004F200000000000130D2000130D3003230C100D0
:100502002D30C2003530C3002030C4007330C50026
:100512006330C6006F30C7007230C8007230C90045
:100522006530CA002030CB006D30CC006530CD0084
:100532006D30CE006F30CF007230D000D10141302B
:10054200D400AF210230D2000130D3002A30C100E2
:100552002030C2006930C3006E30C4007330C50061
:100562006530C6007230C7002E30C8002030C90086
:100572002330CA002030CB006630CC006930CD0079
:100582006E30CE006530CF002E30D000D101413028
:10059200D400AF211030FB003930FC000D30FD00DB
:1005A200FD0BD12AFC0BD12AFB0BD12A0000000043
:1005B200A030B700E030B5000130B6000130B30022
:1005C200B30D33101030B4000D30FC00FB30FD00D1
:1005D200FD0BE92AFC0BE92A00000000F0200130A3
:1005E20083120313D2000130D3002030D400AF2194
:1005F2001F21831203133208103A031D012BF92A1B
:100602003208023A031D092B1030B5070318B60A47
:100612003208053A031D112B1030B502031CB60334
:1006220032080A3A031D172B18238E21E52A20309F
:1006320083120313A0002030A1002030A20020303A
:10064200A3002030A4002030A5002030A6002030D6
:10065200A7002030A8002030A9002030AA002030B6
:10066200AB002030AC002030AD002030AE00203096
:10067200AF00B0010230D2000130D3002030D400EC
:10068200AF21B1011F21831203133208103A031D57
:100692004B2B432B32080B3A031D502B0800310819
:1006A200203E840030303207F000700880000230B3
:1006B200D2000130D3002030D400AF21B10A0A3079
:0C06C20031020318652B432B0800662B47
:04400E00413FFC3FF3
:00000001FF
